:030000000219FDE5
:03000B000200A848
:03002B000201636C
:03005B000202EDB1
:030073000202D3B3
:1000800002030406080C10182030406080040608A3
:100090000C10182030406080A0C000070F1F3F05E3
:1000A000050D050305030302C2AFC0D0C0E0206206
:1000B00017E5256002E473E525F4F58A758B00D217
:1000C00062D0E0D0D0D2AF3285268AC262E526F473
:1000D0006035306803207210758B00D0E0D0D0C23C
:1000E000B1C287C281D2AF32C2B1C287C281206E93
:1000F0000C206609740AD5E0FDE57E4280758B0010
:10010000D0E0D0D0D2AF32758A00C28DD26201FD6C
:1001100001B7306805206602D2B101B7306805200A
:100120006602D28701B7306805206602D28101B726
:10013000C28230680A2066077408D5E0FDD2B1019A
:10014000B7C28630680A2066077408D5E0FDD287FA
:1001500001B7C28030680A2066077408D5E0FDD276
:100160008101B7C2AFC2AD53E6EFC0D0C0E0D2D379
:10017000D2AFC2CEE52A6007207449152A21C4787F
:1001800000790020742EE580307E01F430E502789D
:10019000FF53DACF207E0343DA20307E0343DA10A8
:1001A000C2D8C271E580307E01F430E50279FFC328
:1001B000E89970CB306103752A18207403752A18EA
:1001C000885FD27020740DE52B6004152B21D44379
:1001D000DA01C2D82070024136A85F206102C270E5
:1001E000207431C3E894F0400374F0F8E8C4540F6D
:1001F00028F87984B703024114C313C3138721205D
:100200000802C313200A06C3C898F8411428F850FE
:100210000374FFF8C3E895685003E568F88822E5A1
:100220002D54066011E533C313C31324062522F5AC
:100230002250037522FF852224A824C3E524956457
:100240004002A8648825E5697002417AC3E8AA697A
:100250009A5003E8FAE4F9EAC333FBE56BF45B294F
:10026000400D256AF8E56A6002156A400B417A0A7A
:10027000C3E56A9A5002056A78FF8826C26EC3E514
:100280002694F84002D26EC3E52594404002D26421
:1002900020CF0AD0E0D0D043E610D2AD32C2CF0595
:1002A0003A7801E52A6005307402152AC3E55F94A7
:1002B00001400575620041C9756300756C00E56217
:1002C0002401F56250037562FFD0E0D0D043E61000
:1002D000D2AD32C2AFC0D053E67FC2607591008507
:1002E0005694855795759104D0D0D2AF32C2AF5392
:1002F000E6EFC2ADC0D0C0E0C0F0D2D3D2AFA8FB11
:10030000A9FCC2D8307102615453DACF207E034376
:10031000DA10307E0343DA20D271E580307E01F4BA
:1003200020E502612B88278928A18153DACF207E1E
:100330000343DA20307E0343DA10C2D8C27130742E
:1003400002A16D7800E580307E01F430E502A16DF8
:10035000885FA15553DACF207E0343DA20307E0335
:1003600043DA10C271206102812D53DACF207E035F
:1003700043DA10307E0343DA20C2D8D271885A891A
:100380005BC3E89558F8E99559F97B007E087A0037
:10039000C3E8948CE994005005755E00811F8821A4
:1003A00078A2E6A8216055C3E894C8E994005008F3
:1003B000E4D2E4FB7A0A61FAC3E89468E994015054
:1003C00008E4D2E3FB7A0F61FAC3E894D0E994021F
:1003D0005008E4D2E2FB7A1E61FAC3E894A0E994E3
:1003E000055008E4D2E1FB7A3C61FAC3E89498E94D
:1003F00094085008E4D2E0FB7A787E00C3E8955C6C
:10040000FCE9955DFD30E70AECF42401FCEDF434E1
:1004100000FD755E00C3EC9AED9E5003755E018889
:100420005C895D855A58855B597802A155C3E8956A
:1004300027F8E99528F9307C02A139307B02A139EF
:10044000307A02A1322075028150E9FDE8FC816F0B
:10045000E9C313F9E813F8307902A132E9C313F9BB
:10046000E813F8307802A132E9C313FDE813FC2049
:0E047000612CC3EC941CED940240028186EDD9
:10047E00701EC3EC94C850180529E5297002152981
:10048E00C3E529940A5002A16D755F00D270A16D6B
:10049E00E529600215297888E6F97400207F08782E
:1004AE0096B90302789EE624FAFEE43400FFC3EC0C
:1004BE009EFCED9FFD9208B90310A208500720760E
:1004CE0009D27681D8307602C276A2085016B903C8
:1004DE000DECF42401FCEDF43400FD0204F278007E
:1004EE007900A139B90315EC33FCED33FDC3EC945F
:1004FE000AFCED9400FD50047C007D00C3EC94FFDB
:10050E00ED9400400678FF7900A139EC8575F0A4D2
:10051E00C5F0A2F733F87900400302055578FF794C
:10052E0000020555E9C313F9E813F8307C0EE960B3
:10053E000278FFC3E81338F8E43400F9C3E894FFF7
:10054E00E99400400278FF885FD270206102A16DAD
:10055E00741FF4552F4BF52FC274EB7002D27475C5
:10056E002A18307403752A0A306102A1812074039F
:10057E0053DAFE207403752B06D0F0D0E0D0D0D223
:10058E00AD43E6103279010205B179030205B17966
:10059E000A0205B1791E0205B179640205B179C866
:1005AE000205B17817E4D5E0FDD8FAD9F6227A140F
:1005BE007B780205D87A107B8C0205D87A0D7BB435
:1005CE000205D87A0B7BC80205D87902B27DE4C247
:1005DE0086D5E0FDD287D5E0FDC287D5E0FDD28677
:1005EE00D5E0FDD2B1E576D5E0FDC2B17496D5E089
:1005FE00FDD9D9EAF8D5E0FDD8FBDBCEC28622C301
:10060E007C007D0075F00005F0EA33FAEB33FB5009
:10061E00F6EB13FBEA13FAC3E9FFE8FEE89AF8E9F2
:10062E009BF95004EFF9EEF8B3EC33FCED33FDD546
:10063E00F0DFEDF9ECF822E889F08A20D2D4F8A99F
:10064E00F07B0030F70B7BFFF42401F8E9F4340063
:10065E00F9E88520F0A4ADF0F8E98520F0A4AFF01C
:10066E00FEED2EF974003FFA7C04C3EA13FAE91387
:10067E00F9E813F8DCF48BF030F70AE8F42401F80B
:10068E00E9F43400F9E889F0C2D4F8A9F02222C3C3
:10069E00E54113F9E54013F8C3E54598F8E54699A9
:1006AE00F9500CC3E89480E994FF40160206D4C3B7
:1006BE00E8947FE9940050030206D4787F79000213
:1006CE0006D4788079FF884A894B22E54A2547F877
:1006DE00E54B3548F9854B20E4300701F43549FAEE
:1006EE0030E709C3EA94F04015020712C3EA940FEB
:1006FE00500302071278FF79FF7A0F020712780073
:10070E0079007AF0C3E5249564500AC374019524E8
:10071E00500B020730E54B20E70E020730E54B3059
:10072E00E706884789488A492278A4E6FAC3E54A4B
:10073E0033F8E54B33F9D145E930E70BC3E8948044
:10074E00E994FF4013E16AC3E8947FE994005002F4
:10075E00E16A787F7900E16A788079FFE820E71511
:10076E00C3E52398F84009C3E894014003020791BA
:10077E007801020791E8F424012523F840030207CB
:10078E009178FF884C2278A5E6FAA848A949D14568
:10079E00E930E70CC3E89401E994FF40160207C55F
:1007AE00C3E894FFE9940050030207C578FF79006F
:1007BE000207C5780179FFE920E715C3E54C98F8E3
:1007CE004009C3E8940140030207EC78010207ECEC
:1007DE00E8F42401254CF840030207EC78FF882446
:1007EE002278FFC26420693D206A12D264C3E541BB
:1007FE00940A4009C3E52594405002C26479A1E7EA
:10080E006023E541601F74FF8541F0848539F03027
:10081E006A0375F005A4F8C5F0600278FFC3E89589
:10082E00675002A867886622C3E5409440E541946C
:10083E0001E5665003140147046002F566220208C2
:10084E004F2275E890227883E6FFE5E820ECF7A8C2
:10085E00BDA9BE0573C3E57394084052757300E9D4
:0D086E00FA79A0E76044EA7007E574601BAA
:10087B0002088AC3E895746010E5745006600C1486
:10088B000208960460F9020896E574F574C394A8FF
:10089B00401B7564C0C394054013756480C39405F5
:1008AB00400B756440C39405400375640075BB062B
:1008BB0022E564F460020564E573B4070375BB1E9F
:1008CB0022743279A687F0A4C5F0A2F733F8C3E8F7
:1008DB0095644002A8648822882488258826886726
:1008EB00227540007541F022C2AF75C820A8CCA973
:1008FB00CDAA3A30CF010A75C824D2AFAB3BAC3C82
:10090B00883B893CC3E89BF8E99C206908F9306770
:10091B000241082165AD3D8A3DF9EA9DFA600478F4
:10092B00FF79FFAE3EAF3F8B3E8C3FC3EC9FFCC3CA
:10093B00E99CF542A83BA93CC3E89EF8E99FF9C3A3
:10094B00E54113FBE54013FAE82AF540E93BF54195
:10095B0050067540FF7541FF21AFAA40AB41AC403B
:10096B00AD417E047F02C3EB940440021E1FC3EB18
:10097B00940840021E1FC3ED13FDEC13FCDEF7C3FE
:10098B00EA9CFAEB9DFBEF6009C3E913F9E813F856
:10099B00DFF7EA28FAEB39FB8A408B4150067BFFE5
:1009AB008B408B41C3EB94025002D2673069047FBA
:1009BB000321DA7892E6FFC3E537948240110FC327
:1009CB00E53794A040010FC3EF940640027F057EEC
:1009DB0005E541C4540FF9E541C454F0F8E540C4B2
:1009EB00540F28F8C3E89EFAE99400FB4009C3EAC8
:1009FB009402EB940050047A02E4FB4154AA40ABFE
:100A0B0041EBC4FEEAC4540F4EFCC3EA9CFAEB94D0
:100A1B0000FBC3E813C313F8EA28FAEB3400FB8A94
:100A2B00408B41C3EB94024002C2677805EBC4FED6
:100A3B007B00EAC4540F4EFAC3EA98FA4005C394FC
:100A4B000250027A027892E6FF30600241548552DE
:100A5B0056855357D26043E680C3E49AF8E49BF97A
:100A6B0030670241EEE8FAE9FBD3E913FDE813FC2A
:100A7B0088528953C3EF94036038EF20E00DE82CC4
:100A8B00F8E93DF9ECFAEDFB020AA9E828F8E93997
:100A9B00F9C3E82402F8E93400F97AFE7BFFC3EFCF
:100AAB009403400E8A548B55884E894F8C508D5130
:100ABB006122885489558A4E8B4F8C508D513069E9
:100ACB0020C3E53394034019E542A2E713F8E5553B
:100ADB00F4240138400B20E7087554FFF42401F58A
:100AEB00556122E8FAD3E813FC8852C3EF940360F4
:100AFB0020EF20E007E82CF8ECFA610EE82824023E
:100B0B00F87AFEC3EF940340088A54884E8C5061E8
:100B1B002288548A4E8C50E56BC3335002646BF5BC
:100B2B006B306002612C753402D26043E680E52D98
:100B3B0054066026A840A941C3E913F9E813F8C28B
:100B4B00AF53E67F759100C3E498F594E499F5955E
:100B5B00759104D26043E680D2AF22D26575440012
:100B6B00752000306B03752040020B85D2657544F0
:100B7B0000752040306B03752000D2AF78012067E1
:100B8B0022E52D54066002C265C3E541940540136E
:100B9B007802940540087803940540027806306982
:100BAB0002780A206019E544601530690AC3E53301
:100BBB0094034003D53406D2AFD26C81567134D234
:100BCB00AF0000C2AF206726E541C3FB940F400284
:100BDB007B0FEB240530730123306A0274282062EB
:100BEB000123F93069027982E58BC39940B505443D
:100BFB00E59B5440B52002814030690A08C3E89454
:100C0B000A40010861AE2065026185C26553E67F2B
:100C1B007591003067107594007595FE759104D22F
:100C2B006043E6806185AE40AF41C3E49EF594E43A
:100C3B009FF5958127C3E53394025002618530659A
:100C4B00026185D802815461AEC26C53E67F759107
:100C5B0000855494855595759104854E56854F574F
:0D0C6B00D26043E680D2AFE52D540660084C
:100C7800206A020533020C90306C0D206B0A206547
:100C8800071581158102151F22780030640530652B
:100C9800027801E53775F007A4F9E5F028F5F0E9E1
:100CA800A2F013A2F113A2F213F537C394785003FC
:100CB800753778C3E53795384008D266C2B1C28720
:100CC800C28130600281CA855056855157D260432F
:100CD800E68022207D11C2AF754302C286D282D23D
:100CE800AF759F02020EAAC2AF754302C286D280B8
:100CF800D2AF759F02020EAA307243207D20C2AF88
:100D0800754303900141757E40C281C28030620400
:100D1800D287A11ED286D2AF759F03020EAAC2AF98
:100D2800754303900141757E40C2B1C282306204AE
:100D3800D287A13ED286D2AF759F01020EAA207D2E
:100D480017C2AF75430390011CC281306202D2877B
:100D5800D2AF759F03020EAAC2AF75430390011C60
:100D6800C2B1306202D287D2AF759F01020EAA20AB
:100D78007D11C2AF754304C282D280D2AF759F0184
:100D8800020EAAC2AF754304C280D282D2AF759F49
:100D980003020EAA307243207D20C2AF754305902E
:100DA8000130757E04C287C286306204D2B1A1BA0E
:100DB800D282D2AF759F02020EAAC2AF75430590C8
:100DC8000152757E01C287C286306204D281A1DADF
:100DD800D280D2AF759F02020EAA207D17C2AF75CE
:100DE8004305900112C287306202D2B1D2AF759F1B
:100DF80002020EAAC2AF754305900126C28730626F
:100E0800EBD281D2AF759F02020EAA207D11C2AF2C
:100E1800754306C280D286D2AF759F03020EAAC25E
:100E2800AF754306C282D286D2AF759F01020EAA61
:100E3800307242207D20C2AF754301900152757E09
:100E480001C2B1C282306204D281C156D280D2AF0F
:100E5800759F01020EAAC2AF754301900130757EDD
:100E680004C281C280306204D2B1C176D282D2AFCC
:100E7800759F03C1AA207D16C2AF75430190012654
:100E8800C2B1306202D281D2AF759F01C1AAC2AF8E
:100E9800754301900112C281306202D2B1D2AF759E
:100EA8009F03C26622900110757E00C2B1C287C23C
:100EB80081C282C286C280C26222788076FF0876AA
:100EC800FF0876FF0876FF08760308760408760997
:100ED800087603087601087601788C76010876FF93
:100EE8000876FF0876FF0876FF0876FF087603087D
:100EF80076FF0876FF0876FF0876250876D008760C
:100F0800FA0876FA0876040876FF0876010876006B
:100F180008767A0876FF08760108760108760008D0
:100F28007603227887E6FFC272BF0302D2727888FE
:100F3800E6C394036008C27DE630E102D27DC27E3A
:100F48007889E630E102D27EC3EF94026008758E9C
:100F580001D273020F63758E00C273227880E61483
:100F68009000809378A4F67881E6149000809378B6
:100F7800A5F67886E61490008D9378A6F6789CE618
:100F88007538FF75390CB402067538A075390AB47E
:100F9800030675388275390578A3E61490009A938C
:100FA800F569D1AD22227896E6FA7897E6FB78883B
:100FB800E6B40305C3EB940EFB307F047A007BFF95
:100FC800C3EB9AFCC3948250027C82757500057548
:100FD800EC8575F0A4C3E5F0947D40F222D27FF150
:100FE800AE1205A27A007B007C10120598E55F2AF4
:100FF800FA74003BFBDCF37C04C3EB13FBEA13FA43
:10100800DCF7FEC27F120FAE22E5EF20E603752063
:10101800000520903DFFE520146006901FFF146036
:10102800009304600375EF1253D9BF7581C043FF65
:101038008012059375EF0243B203E5B3240420E759
:101048000DF521E5B120E0068521B343B101120E6B
:10105800AD75803875A4C775F1FF75D4DF7590FF3D
:0F10680075A50075F20075D50075A0FF75A6007F
:1010770075F30075D60075B0E475A71B75F4FF7599
:10108700E241E4F8F6D8FD756B01120EC212156144
:1010970078988676753001C2AF1205AC1205BC127E
:1010A70005A21205C31205A21205CA1205A212163D
:1010B7007A1205AC1205AC1205A7C2AF78FA79FA15
:1010C700308507D9FBD8F7021C00120F2B120F64CB
:1010D700120FAD120FAE78988676120EAD75885046
:1010E70075891275C82475910475D84075A822753D
:1010F700B80275E690759B80759D0075D10E75BC1D
:101107005875BB0675BA1F75E880120593D2AF12E2
:10111700084C53DACF207E0343DA20307E0343DACC
:101127001043DA01C2D8C2711205ACD2617B037ACF
:101137000CE55E70077A0CDB030210C11205A220D2
:1011470070030210C1C270E55FC3940240E1E52F4E
:10115700541F856160F561B560D5DAD5C26153DA90
:10116700CF207E0343DA20307E0343DA10C2D8C291
:101177007178A2E67008D274E52F54E0F52FC27596
:101187007529001205A7307409C3E529940A40029E
:10119700D27512059878023074027800C3E55F981B
:1011A70040F0C2AF1205BC1205BC1205BCD2AF128B
:1011B70005AC754D007888E6B4030241A112059885
:1011C700788CE6C3940150030212A1E530C3940161
:1011D70050030212A1207435C3E55F94FF50030248
:1011E70012A1C2AF1205D1D2AF1205A7C3E55F9412
:1011F7000150EFC2AF1205BC12059D1205BCD2AF5C
:101207001205A7C3E55F94FF40E90216FF7F05D2E9
:101217007F120FAE1205A7C2AFC27F120FAEAE5F2D
:10122700C3E55F947FD2AF407B120593C2AF12052F
:10123700D1D2AFDFDA120FE5C3EE94057897F61235
:1012470005AC1215A31216827F0AD27F120FAE12B7
:1012570005A7C2AFC27F120FAEAE5FC3E55F947F33
:10126700D2AF50E4120593C2AF1205BC12059D120E
:1012770005BCD2AFDFD4120FE5EE24057896F6123F
:1012870005AC1215A31216B11205A7120FAEC3E5CE
:101297005F94FF500221DC0216FFC3E55F954D40C6
:1012A70003855F4D1205A778017988E7B4030278B3
:1012B70005C3E55F98400221BCC2AF1205D11205F4
:1012C700D11205D1D2AF1205AC753000E4F531F576
:1012D700320531E531F470390532789AE678191418
:1012E7006012783214600D787D14600878FA146003
:1012F70003753200C3E53298401715327531B4785B
:10130700998676C2AF1205D1D2AF78988676120544
:10131700A712059DE52A700530740201C1780120E6
:1013270074027806C3E55F9840A77888E6C39403FC
:1013370060031205A7E52A70030210C1C2AF120E9F
:10134700ADE4F522F523F524F525F526F56AD2AFA8
:101357007885E6C333F568E4F545F546F547F5487E
:10136700F549F573F52CF52DF53775730875BB1E23
:10137700120593120850E5E820ECFBA8BDA9BEE9C9
:101387007001F8887412085475730875BB1E788746
:10139700E6FE7602120F2B7887EEF6C2AF7564FF72
:1013A7001208CC852264852265852266D2AF752214
:1013B7000175240175250175260185636C756D011D
:1013C7007888E6B40307C27D307602D27DD268D230
:1013D70069753300120E13120E381208EC1208F357
:1013E7001208EC1208F31208EC021400C2AF120F35
:1013F7002BD2AF75730075BB06120B7712069C12C2
:101407000C91120CDB1208F3120B66306D031206F7
:101417009D2067031207EF306703120836120C91FD
:10142700120D001208F3120B77306D031206D91252
:101437000C91120D771208F3120B66306D03120729
:1014470037120C91120D9C1208F3120B77306D03B3
:10145700120794120C91120E131208F3120850126D
:0E1467000B66120C91120E381208541208F384
:10147500306932206B2F85676485676585636C7578
:101485006D0179187A0CC3E53399400CC269D26AAB
:101495008A357564FF0214AAC3E55F94014003020F
:1014A5001400021527306A1B206B18E535147004EB
:1014B500C26A61F3F535C3E55F9401400302140088
:1014C500021527753600C3E562788298505430744A
:1014D50004E52A604D7888E6B40317207D0520765B
:1014E5000781F730760281F7206B07D26B85676439
:1014F500813F78F0306B058567647820C3E54198B6
:1015050050028100306B1BC26BC27D307602D27DEA
:10151500D26A75351285676481000536E55F60021C
:10152500A12A753600C2AF120EAD7887E6FE7602A7
:10153500120F2B7887EEF6E4F522F523F524F52531
:10154500F526F568C268D2AF120593120EAD307458
:1015550009C3E5369405400201C141D3901A0D78BF
:10156500201215E5E520B45A0CA31215E5E520B4C3
:10157500A503021583120EC21215A30215A2901A15
:101585000378807B0A1215E5A308DBF9901A0F781A
:101595008C7B181215E5A308DBF9901A2722C2AF38
:1015A5001216241215FE901A00740E1215EAA37471
:1015B500041215EAA374141215EA901A0378807BB5
:1015C5000A1215E9A308DBF9901A0F788C7B18121B
:1015D50015E9A308DBF9121637121615901A2722FA
:1015E500E493F622E6438F01538FFD75EF0275B73D
:1015F500A575B7F1F0538FFE22438F02438F017516
:10160500EF0275B7A575B7F1901A0DF0538FFC224F
:10161500901A0D745AB1EA901A0E74A5B1EA227A9D
:101625003079D07820901A40B1E5E520F709A3DAA2
:10163500F7227A3079D0901A40E7B1EA09A3DAF9AE
:1016450022AB77A878BB01027984BB02027985BBFE
:1016550003027986BB04027992BB05027987BB0632
:101665000279A3BB0702799CBB08027988BB0902F2
:101675007989E8F7227C051205ACDCFB22C2AF12A2
:1016850005BC1205C31205CA1205D112059D120526
:10169500BC1205C31205CA1205D112059D1205BC5F
:1016A5001205C31205CA1205D1D2AF22C2AF120567
:1016B500D11205CA1205C31205BC12059D1205D12A
:1016C5001205CA1205C31205BC12059D1205D112D9
:1016D50005CA1205C31205BCD2AF22AE77AF78C2D8
:1016E500AF1205BC1205BC1205BC12059DDEF21237
:1016F50005D112059DDFF8D2AF22D182D17AD17AF8
:10170500757701757801757900D1E07C05AD5F12BB
:1017150005ACC3ED955F70F5C3E55F9401400AC361
:10172500E55F94FF403202173BD146B1A3D182C297
:10173500AF75EF12D17ADCD50579C3E579940350FD
:101745000280C6D17A0578E5771490009F93F80852
:10175500C3E57898500280AED17AD17A0577C3E592
:1017650077940A5002809C120EC2B1A3C2AF75EFE6
:0317750012D17A14
:0319FD00021011C4
:101A00000E0414FFFFFFFF0304090301015AA5019F
:101A1000FFFFFFFFFF03FFFFFF25D0FAFA04FF01DE
:081A2000007AFF01010003FF41
:101A4000235475726E696779343041232020202039
:101A500023424C48454C4923463331302320202033
:101A60002020202020202020202020202020202076
:101C0000C2AFC2D353D9BF7581C043B20343FF8073
:101C1000752438752503B1C975EF0275E24043F1AB
:101C20002053A4DF75D400D2857DFA780379E67C51
:101C300010752200752300901DD67B0675249875BB
:101C400025013085028142208508D8FBD9F9DCF7CF
:101C500081B4308508D8FBD9F9DCF781B4B189E4C7
:101C600093A3C39A6004DDC381B4DBDBB17B600264
:101C7000812B7B08E493FAA3B15CDBF87A30B15C8A
:101C8000752200752300B17BEAFCEBFDC3ED94FEE9
:101C9000400EB17B8A278B28ED30E0048A828B834B
:101CA000B17B7AC270D8C3ED94FE601350CEBD00F4
:101CB00025EC60097520007521FF0200008100A855
:101CC00027A9280809D804D90281D3B17FEA89AAB3
:101CD000F281C50D81A0C3ED94035049EDA2E092BD
:101CE000007AC5C3E5829400E583941C50902000DF
:101CF00010438F02438F0175B7A575B7F1F030001F
:101D00001FA827A9280809438F01538FFDD804D99C
:101D100002A12089AAE275B7A575B7F1F0A3A10DBC
:101D2000538FFC817C7AC1BD030CE493A3FAB140CC
:101D3000DCF8B138817C817EAA22AB23B15CEBFA5E
:101D4000EA6222752608C3E52313F523E52213F57D
:101D50002250066323A0632201D526EAB1C9B1C986
:101D600075260AEAF4200102D285300102C285B14B
:101D7000C9C3134002C201D526EB22B17FEAFB2082
:101D80008502A17F308502A184752608AE24AF2587
:101D9000C3EF13FFEE13FEB1CDB1C9C3EA13308513
:101DA000024480FA30E703632201C3E52313F523DD
:101DB000E52213F52250066323A0632201D526D91C
:101DC000E52265236523F52222AE24AF250E0FDE22
:101DD000FEDFFCD20122424C48656C693437316326
:041DE000F3100601F5
:00000001FF
